S31501A0000004F01FE5E067A001F8B504000D00160095
S31501A00010002701F097FF002007003800310080B2C9
S31501A0002089B2884208D20122BFB2E95914FA87F0EF
S31501A0003002F002F83F1DF0E7B6B2042096FBF0F1FC
S31501A0004000FB1160002806D00122BFB2E95D14FAB7
S31501A0005087F001F0F1FFF1BD10B5040000212000E9
S31501A0006002F04EF910BD01000020C9B201291DD030
S31501A00070C9B202291AD0C9B2032917D0C9B2052912
S31501A0008014D0C9B2102911D0C9B281290ED0C9B2D2
S31501A0009083290BD0C9B2852908D0C9B2902905D028
S31501A000A0C9B2D02902D0C9B2D12901D101221000E9
S31501A000B0C0B270470100C9B201291DD0C9B2022937
S31501A000C01AD0C9B2032917D0C9B2052914D0C9B209
S31501A000D0102911D0C9B281290ED0C9B283290BD05A
S31501A000E0C9B2852908D0C9B2902905D0C9B2D029EB
S31501A000F002D0C9B2D12900D10800C0B2704710B54B
S31501A001000400E4B2002C14D1DFF8880C007B00288F
S31501A001100BD1DFF8800CC07950F04000DFF8C41C89
S70501A0667C77
